:100000005AC073C072C071C070C06FC06EC06DC086
:100010006CC06BC06AC06AC068C067C066C065C09B
:1000200064C063C062C040C3FFC20DC313C318C322
:100030001EC33FC33EC33DC32EC338C337C336C3FD
:1000400035C334C333C332C331C330C32FC32EC30C
:100050002DC32CC32BC32AC329C328C327C326C33C
:1000600025C324C323C322C321C320C31FC31EC36C
:100070001DC31CC31BC31AC319C318C317C316C39C
:1000800015C314C313C312C311C310C30FC30EC3CC
:10009000C4C20CC30BC30AC3ADC208C307C306C3A3
:1000A00005C3A5C2BEC202C301C3B5C2FFC2FEC220
:1000B000FDC2FCC2B4C211241FBECFE5D4E0DEBF36
:1000C000CDBF11E0A0E6B0E0EAEBF6E002C005909B
:1000D0000D92A43EB107D9F712E0A4EEB1E001C041
:1000E0001D92AC3BB107E1F765C28ACF1F920F9218
:1000F0000FB60F9211242F938F939F93EF93FF933B
:100100005C9B02C084E00AC02CB190913302973707
:1001100011F0109276025B9B04C083E08093320260
:100120001DC0809131028B3418F083E68093320237
:1001300080913102E82FFF27EC51FE4F2083973743
:1001400029F4809131028F5F80933102973731F427
:1001500080913102813410F010927602FF91EF917C
:100160009F918F912F910F900FBE0F901F90189518
:1001700088E98AB983E389B910922F02109230027C
:100180001092310208955D9BFECF8CB90895000056
:10019000000000000000000000000000000000005F
:1001A000000000000000019791F708950000000092
:1001B00008958FB9779BFECF08951F93CF9384E165
:1001C0008DB987E387BB10E080E288BBEFDFC5987D
:1001D000EDDFC59AEBDFC12FC598E8DFC59AB3996B
:1001E0001160C73008F4110FCF5FC830A8F3DEDF0D
:1001F000C598DCDFC59ADADFC598D8DF8FE387BB07
:1002000080E288BBD3DFC59884E58DB9812F99271B
:10021000CF911F910895982F85E08FB9779BFECFDE
:10022000905E9FB9779BFECFC8DF992708950F9303
:100230001F93182F062F84E0BCDF812FBADF802F99
:10024000B8DF80E0B6DF1F910F910895AC0120E088
:10025000261750F4FA01E20FF11D80818FB9779BC8
:10026000FECF2F5F2617B0F3089584E18DB918BA39
:1002700087E187BB1BBC81E08ABD80E48FBD89E03C
:100280008EBDB39BFECFB399FECF1FBC1EBC18BA68
:100290008FE387BB84E58DB98AE090E078DF08952D
:1002A00063E084E291E0D2DF64E288E291E0CEDFB5
:1002B000DCDF08950F931F93CF93C0E005E312E0B6
:1002C000C05EF80161918F018C2FB1DFCF51C03436
:1002D000B8F3CF911F910F9108950F931F93CF9370
:1002E000C0E005E312E08C2F8058F80161918F0186
:1002F0009EDFCF5FC034B8F3CF911F910F91089567
:100300000F931F938C0163E084E291E09FDF602FE5
:100310008AEF8DDF64E28DE491E098DFA6DF1F9124
:100320000F910895682F8AEF82DF64E282E791E0FF
:100330008DDF9BDF089563E084E291E087DF64E274
:1003400087E991E083DF91DF08950F931F9367E2C0
:100350008CEB91E07BDF89DF62E08FE191E076DF7B
:100360002CDF9927182F002762E081E291E06EDFF1
:1003700024DF9927082B192BC8011F910F9108958D
:10038000A89A8EE190E003DFA8988EE190E0FFDE6E
:1003900060E380E690E05ADF68DF67E281E990E0A1
:1003A00055DF63DF69E389EB90E050DF67E283EFBD
:1003B00090E04CDF5ADF62E08BE191E047DFFDDE49
:1003C0008093BB0262E08DE191E040DFF6DE809336
:1003D000790284EF91E0DBDE62E08BE191E036DFD1
:1003E000ECDE8093BB0262E08DE191E02FDFE5DE81
:1003F0008093790208950F931F93CF93DF93809199
:10040000BB028823B9F480917902853098F400E02A
:1004100010E0C80187DFC0E0D0E08C2FFCDEB3DE47
:100420002196C034D105CCF30F5F1F4F0F3F11054C
:1004300081F37CF381E0809376028FE68093330230
:10044000DF91CF911F910F910895AF92BF92CF92FC
:10045000DF92EF92FF920F931F93CF93DF938FE67C
:1004600092DE81E080937602809176028130E1F322
:100470008091E401A82EBB2481E080937602109243
:100480003102109234028091BB02882309F069C0C6
:1004900080917902853008F064C002DFCC24DD242D
:1004A0008FE671DE81E080937602809131028034A4
:1004B000E0F3E5E3F2E0A4EEB1E09F01215C3F4F01
:1004C0008D9181932E173F07DCF7F4DEC60118DF0C
:1004D000C60128DFC0E0D0E045E3E42E42E0F42E80
:1004E0000AE712E08C2F97DE982FF80181938F0195
:1004F000F70181917F01891709F000002196C0342E
:10050000D10584F3C0E0D0E035E3E32E32E0F32EF2
:100510000AE712E08C2F7FDE982FF80181938F017C
:10052000F70181917F01891719F081E080933402EE
:100530002196C034D10574F31092310237DE08944D
:10054000C11CD11CAC14BD040CF0AACF80913402A4
:10055000882311F48FE601C088E715DE8FE68093CB
:100560003302DF91CF911F910F91FF90EF90DF90B9
:10057000CF90BF90AF900895A89A8EE190E007DEEB
:10058000A8988EE190E003DE08958FE387BB9FEF8C
:1005900094BB91BB18BA15BA12BA84E58DB9A89A62
:1005A0009093BB02909379021092340281E0809381
:1005B00076020895CFE5D4E0DEBFCDBFE6DFD8DD1B
:1005C0007894909176029923E1F78091E4018093E9
:1005D0003302909331029927AA27BB27FC01F09799
:1005E000E834F10508F062C0ED5EFF4F0994C8DE03
:1005F0008EE60FC062E08BE191E028DEDEDD8093C5
:10060000BB0262E08DE191E021DED7DD80937902CB
:10061000805DB9DD4BC0EFDE49C042DE03C015DFAF
:1006200045C0AC988FE6F5CFA89A8EE190E0AFDD9B
:10063000A8988EE190E0ABDD60E380E690E006DE16
:1006400014DE81E326C067E281E990E0FFDD0DDE84
:1006500082E31FC069E389EB90E0F8DD83E319C012
:1006600067E283EF90E0F2DD00DE84E312C062E037
:100670008BE191E0EBDDA1DD8093BB0262E08DE1D7
:1006800091E0E4DD8EE190E082DD97DD80937902F8
:1006900085E379DD0EC0A89A8EE190E078DDA89818
:1006A0008EE190E074DD05C0A89803C081E08093DE
:0A06B000760281E08093760284CF89
:1006BA0032800000000000000023D90037B800375C
:1006CA00B04027C1D027C85837A80037A01827D963
:1006DA000037C98037D20037804037C0001BFC483A
:1006EA003037B80037B04027C1D027C85837A800DC
:1006FA0037A01827D90037C98037D20027D0083742
:10070A00803037C00037F8902737B80037A018373D
:10071A00A80037B04037C28837CFE037D18037FFDB
:10072A009000000037B80037A01837A80037B0404B
:10073A0037C30037CF5037D18037B88037F89000A9
:10074A0000003937B80037B04027C1D027C858371A
:10075A00A80037A01827D90037C98037D20027D078
:10076A000037803037C00037F8902705F805F917A9
:10077A00E417E00227E0680337B80037B20027C160
:10078A00D027CA1837A80037A01827DC0037C98035
:10079A0037D20037802837C00037F8902437B8009E
:1007AA0037B04027C1D027C85837A80037A0182724
:1007BA00D90037C98037D20037801037C00037F8E0
:1007CA00902437B80037B04027C1D027C85837A877
:1007DA000037A01827D90037C98037D200378008D8
:1007EA0037C00037F8902437B80037B20027C1D095
:1007FA0027CA1837A80037A01827DC0037C980375E
:10080A00D20037802037C00037F8902437B8003735
:10081A00B04027C1D027C85837A80037A01827D911
:10082A000037C98037D20027D00037803837C00058
:04083A0037F89027D4
:00000001FF
